:020000040000FA
:060000000219FD0200C818
:03000B0002008D63
:03002B000200923E
:03005B000202CBD3
:030073000200B5D3
:100080000406080C10182030406080A0C0C28D0506
:100090004032C0D0C0E0C2CF0541E5646009E563ED
:1000A000600575630001B0756301E52360021523E7
:1000B000D0E0D0D032C2AF53E67F7592FA7593FF8D
:1000C000C22053917FD2AF32C2AF53E6EFC0D0C04F
:1000D000E0C0F0D2D3D2AF5388EFA88AA98CAA404F
:1000E000308D010A758A00758C00754000438810B8
:1000F000E564700AC3E833F8E933F9EA33FA3033D8
:100100001FE8C4540FFAE9C454F04AFAC3132AFA98
:10011000C3E833F8E933F9E82AFAE93406FB217336
:1001200030320FC3E833E933FAE82AFAE93400FB46
:100130002173303115E875F056A4AAF0E975F05630
:10014000A42AFAC5F03400FB2173C3EA13FAE913B9
:10015000F9E813F8E875F056A4AAF0E975F056A48A
:100160002AFAC5F03400C313FBEA13FAC3EB13FBFE
:10017000EA13FAC3EB94125006C3EB9406501A0527
:1001800022E52270021522C3E522940A500241BEE4
:100190007552007A007B00418CE522600215223006
:1001A00035067C007D0821B3AC31AD32303A04AC69
:1001B00033AD34C3EA9CFAEB9DFB9208AE5EAF5FB1
:1001C000303A425007203409D23421D1303402C2AF
:1001D00034303404AE60AF61203902B234C3EA3344
:1001E000FAEB33FBA208500AEAF42401FAEBF434E8
:1001F00000FBC3EA9450FAEB9400FB501478007AA9
:10020000007B004111A208500878007A007B004171
:1002100070E5255403601B202A18E55B33F9EB7069
:1002200007C3E99A4002E9FAE53CC4332AFAEB3401
:1002300000FBEA8EF0A4F9AAF0EB8EF0A42AFAC52E
:10024000F03400FBC3EB13FDEA13F8C3ED13FDE834
:1002500013F80FEF146004C3E833F8C3E933EA334B
:10026000FAEB33FBDFEDEB30E30678FF7AFF7B0739
:100270008852D230C3E559FC955A4002AC5AC3ECBF
:1002800095525008EC75F008A4FAABF0EAF4F8EBDC
:10029000F45407F9C3E89432FAE99400FB50047A65
:1002A000007B00885489558A568B5775230AD0F0F5
:1002B000D0E0D0D053F7DF43F74043E61032752348
:1002C0000AD0F0D0E0D0D043E61032C2AF53A8FE3F
:1002D000C0D0C0E0D2D3A8F9E55830E20AE5FA2050
:1002E000E24220E13F41EFE5FA30E23820E135C358
:1002F000E55513F8E55413F5E988EAC3E55713F813
:10030000E55613F5FB88FC85555853F7BFC3E552F6
:10031000940140057553006124E5532401F55350C1
:10032000037553FF53F7DFD0E0D0D043A801D2AF1D
:10033000327901801479038010790A800C791E804B
:10034000087964800479C880007817E4D5E0FDD886
:10035000FAD9F6227A147B7880127A107B8C800C82
:100360007A0D7BB480067A0B7BC88000E562D5E00D
:1003700001227902E4D291D5E0FDD294D5E0FDC20C
:1003800094D5E0FDC291D5E0FDE920E002D29530A0
:10039000E002D293E562D5E0FDE920E002C29530AB
:1003A000E002C2937496D5E0FDD9C9EAF8D5E0FD24
:1003B000D8FBDBB8D2912278FF20282879A1E7600A
:1003C00023E548601F74FF8548F084853FF030299D
:1003D0000375F005A4F8C5F0600278FFC3E8955BEB
:1003E0005002A85B885A22C3E54794A0E5489400D0
:1003F000E55A50031461F8046002F55A2275E8903A
:1004000022055CC3E55C9408405330EDF4A8BDA917
:10041000BE755C00E9FA79A0E76041EA7006E55D27
:100420006018800CC3E8955D600EE55D5005600ABC
:100430001480070460FA8002E55DF55DC3956740AE
:100440001B7559C0C394044013755980C39404406C
:100450000B755940C39404400375590022E5592493
:1004600010500274FFF55922743279A687F0A4C5A2
:10047000F0A2F733F8C3E895594002A859885B22E7
:100480007547007548F022C2AF75C800A8CCA9CD49
:10049000AA4130CF010A75C804D2AFC3EA13FAE902
:1004A00013F9E813F8AB42AC4388428943C3E89B95
:1004B000F8E99C20280A547FF9302C02A1A481FE7F
:1004C000AD448A44F9EA9D547FFA600478FF79FFCD
:1004D000AE45AF468B458C46A842A943C3E89EF87B
:1004E000E99FF9C3E54813FBE54713FAE82AF54706
:1004F000E93BF54850067547FF7548FFA14BAA47F1
:10050000AB48AC47AD487E047F02C3EB9404400D7A
:100510001E1FC3EB940840052029021E1FC3ED13C4
:10052000FDEC13FCDEF7C3EA9CFAEB9DFBEF6009E0
:10053000C3E913F9E813F8DFF7EA28FAEB39FB8A85
:10054000478B4850067BFF8B478B48C3EB94025088
:1005500002D22C3028047F03A1767892E6FFC3E50F
:100560003D948240110FC3E53D94A040010FC3EFBD
:10057000940640027F057E02E548C4540FF9E54821
:10058000C454F0F8E547C4540F28F8C3E89EFAE9CC
:100590009400FB4009C3EA9401EB940050047A01F3
:1005A000E4FBA1F0AA47AB48EBC4FEEAC4540F4EEB
:1005B000FCC3EA9CFAEB9400FBC3E813C313F8EA0C
:1005C00028FAEB3400FB8A478B48C3EB94024002C5
:1005D000C22C7802EBC4FE7B00EAC4540F4EFAC36F
:1005E000EA98FA4005C3940150027A017892E6FF36
:1005F000302002A1F0854E92854F93D22043E680B1
:10060000C3E49AF8E49BF9C3E833F8E933F9302CF2
:1006100002C182E8FAE9FBD3E913FDE813FC884E36
:10062000894FC3EF94036037EF20E00CE82CF8E922
:100630003DF9ECFAEDFB8013E828F8E939F9C3E855
:100640002401F8E93400F97AFF7BFFC3EF940340FB
:100650000E8A508B51884A894B8C4C8D4DC1B6887F
:100660005089518A4A8B4B8C4C8D4D3028127550D5
:10067000F07551FF754CF0754DFF754EF0754FFFDD
:10068000C1B6E8FAD3E813FC884EC3EF94036020A8
:10069000EF20E007E82CF8ECFAC1A2E8282401F8E2
:1006A0007AFFC3EF940340088A50884A8C4CC1B645
:1006B00088508A4A8C4C302002C1B6753A02D2204A
:1006C00043E680E5255403602DA847A948C3E913F4
:1006D000F9E813F8302804E92440F9C2AF53E67F63
:1006E000759100C3E498F594E499F595759104D259
:1006F0002043E680D2AF22D2217549007520003018
:100700002B03752040800ED22175490075204030A2
:100710002B0375200078017901202C20E525540356
:100720006002C2217914E548C313700104F8C39430
:100730001440027814302804781B791BC3E833F87E
:10074000C3E933F9202010E549600C302803D53A7D
:1007500004D223E1CBD1BE0549E59B5440B520022C
:10076000E1B530280908C3E899400118E144202187
:100770000A08C3E8994002E115E144C221C2AF531F
:10078000E67F759100302C127594007595F0759187
:1007900004D22043E680D2AFE115E5487EFFC333A3
:1007A0004009C3334005C3334001FEC3E49E759442
:1007B00000F595E18EC3E53994015002E115302131
:1007C00002E115D802E1C9E144C223C2AF53E67F7A
:1007D000759100855094855195759104854A92854F
:1007E0004B93D22043E680D2AFE525540360072027
:1007F00029020539801030230D202B0A20210715EE
:10080000811581020F042278003021027801E53D34
:1008100075F007A4F9E5F028F5F0E9A2F013A2F1CC
:1008200013A2F213F53DC394785003753D78C3E5E8
:100830003D953E400BD222C295C294C29375D53FDE
:100840003020020140854C92854D93D22043E680B2
:1008500022203810C2AFD291C29075D533D2AF7575
:100860009F322125C2AFD291C29275D51ED2AF75EB
:100870009F322125203811C2AFC29375D52DC29069
:10088000D2AF759F52020925C2AFC29575D52DC250
:1008900092D2AF759F12020925203810C2AFD290B4
:1008A000C29275D52DD2AF759F128079C2AFD29208
:1008B000C29075D52DD2AF759F528069203811C274
:1008C000AFC29475D51EC292D2AF759F3202092570
:1008D000C2AFC29475D533C290D2AF759F320209B0
:1008E00025203810C2AFD292C29175D51ED2AF75F5
:1008F0009F528031C2AFD290C29175D533D2AF75BD
:100900009F128021203810C2AFC29575D533C29195
:10091000D2AF759F12800EC2AFC29375D51EC29121
:10092000D2AF759F52C22222C295C294C293D29076
:10093000D291D29275D53F22788076FF0876FF0853
:1009400076FF0876FF0876FF0876FF0876090876B6
:10095000FF087601788C76010876FF0876FF087626
:10096000FF0876FF0876FF0876030876FF0876FF13
:100970000876FF0876250876D0087628087650088D
:1009800076040876FF0876020876FF08767A0876FD
:10099000FF0876070876010876FF0876FF087600DC
:1009A00008760022FA75F00CA4ABF0EAC333F874B1
:1009B0000133F9E8C333F8E933F9E8C32BF8E93434
:1009C00000F9E8C333F8E933F9227888E6C39403E1
:1009D000D23A5002C23AC238E630E102D238A238E6
:1009E00092397886E6149000809378A6F67886E6A9
:1009F000F53FC394025003753F02789CE6753EFFB5
:100A0000B40203753EA0B40303753E8278A0E6F8F5
:100A1000600674282409D8FCF5677896E631A48826
:100A2000318932789EE631A4883389347897E6316B
:100A3000A4883589363128223035117A007B007C34
:100A4000FF7D007E00519F8B5F8A5E22303A2278C4
:100A500096E6FA7B00789EE6FC7D00C3EA33FAEB6B
:100A600033FBC3EC33FCED33FD7E0A519F8B618A6F
:100A7000607896303A02789EE6FA7B007897E6FC3A
:100A80007D007E00303A10C3EA33FAEB33FBC3EC4F
:100A900033FCED33FD7E0A519F8B5F8A5E2222C3B9
:100AA000EC9EFCED9400FDC3EC9AFCED9BFDC3ECC9
:100AB0009423ED940050047C237D00C3EC94FFED5F
:100AC000940140047CFF7D017BFF0B7A000AEA70F1
:100AD00009C3EC33FCED33FD41CAEC8AF0A4AEF05F
:100AE000ED8AF0A42E947C40E4EAF460DD22D23555
:100AF000513812033D12033D7A007B007C10120333
:100B000035E5522AFA74003BFBDCF37C04C3EB139B
:100B1000FBEA13FADCF7FFEB60027FFFC2355138C6
:100B20002278A5E6F954037000E9540C7000E954EA
:100B3000307000E954C0700022756500756600755C
:100B400097DE7597AD7581C043FF8075EF0675A977
:100B50000031287580FF75F1D175A4007580FF758F
:100B6000D4FF75900775F23F75A53F75900775D551
:100B70003F75A60175E34075E2023128E4F8F6D826
:100B8000FD3138F14578988662753001C2AF1203A5
:100B90004512035412033D12035A12033D1203601F
:100BA00012033D7121C2AF75650075660078FA7950
:100BB000FA308007D9FBD8F7021C0031CA513878C7
:100BC000988662312875A91375A71075C10075A79D
:100BD0000075640075E400758811758E04758909C7
:100BE00075C80475910475D84075D90875F7827574
:100BF0009E0375960075DB4275DA4275A82375E68B
:100C00009075F310759B80759D0075D10C75BCB9FE
:100C100075BB1075E88075B201120331D2AF753C17
:100C200000C230120345C231752200120341C3E5F0
:100C300022940A4024D231C232752200120341C3E9
:100C4000E522940A4013D232C233752200120341C6
:100C5000C3E522940A4002D2331203352030030246
:100C60000BA5C2AF120354120354120354D2AF1295
:100C70000345303A02A117120335788CE6C394017C
:100C80005002A117E530C394015002A1177565A564
:100C90007566F17F02D2355138120341C2AFC235B9
:100CA0005138C3E552947FD2AF406C120331C2AFCA
:100CB000120366D2AFDFDE51EEC3EF7897F6120370
:100CC000451210297F0AD2355138120341C2AFC2F2
:100CD000355138C3E552947FD2AF50E8120331C288
:100CE000AF120354120339120354D2AFDFD851EEBE
:100CF000EF24037896F6F87997E7C3942340039896
:100D00005006E824237897F6120345F17F12105815
:100D1000120341513861A5756500756600120341E3
:100D20007801303A027805C3E5529840028172C2D8
:100D3000AF120366120366120366D2AF1203457543
:100D40003000E4F537F5380537E537F4703E0538FF
:100D5000789AE67819146012783214600D787D1450
:100D6000600878FA146003753800C3E53898401CB1
:100D70003128120331153875370078998662C2AF71
:100D8000120366D2AF78988662120341120339E5E6
:100D900023700261A57801C3E5529840AA1203416D
:100DA000E5237003020BA5C2AF3128E4D2AFE4F50E
:100DB0005CF524F525F53D755C081203311203FD41
:100DC00030EDFDA8BDA9BEE97001F8885D120401EF
:100DD000755C08C2AF7559FF120468855B59855B65
:100DE0005AD2AF75A71075C13075A70075A90375E4
:100DF0006401303A07C238303402D238D22875390B
:100E00000011E131041204801204871204801204DC
:100E10008712048012070711071151120487120666
:100E2000F7202C031203B7302C031203E71107112C
:100E3000741204871207071107119912048712060A
:100E4000F7110711BC120487120707110711E112ED
:100E500004871203FD1206F7110731041204011270
:100E60000487302827855B5979187A0CC3E53999AE
:100E7000400EC228D2298A3B855B59855B5A800C7B
:100E8000C3E55294014003020E14E10C30291C20EA
:100E90002B19E53B147006C229D22AC114F53BC3B5
:100EA000E55294014003020E148061753C0078FA0B
:100EB00079A4E760027803C3E55398504FE52360B7
:100EC0004B303A17203805203407800F3034028029
:100ED0000A202B07D22B855B59C13E78F0302B05B9
:100EE000855B597820C3E548985003020E14302BD7
:100EF0001BC22BC238303402D238D229753B12853E
:100F00005B59C114053CE5526002E10F753C00C21B
:100F1000AF312875240075250075A91375A71075C4
:100F2000C10075A700756400D2AF12034131287863
:100F3000A4E66006C290C291C292C3E53C9404400C
:100F40000261A5A142901A0D7820F1BAE520B455AE
:100F50000AA3F1BAE520B4AA0280063138F17F80F5
:100F60001D901A0378807B0AF1BAA308DBFA901A65
:100F70000F788C7B1AF1BAA308DBFA901A2922C2E7
:100F8000AF120FFDF1DA901A007410F1BFA37403D1
:100F9000F1BFA37421F1BF901A0378807B0AF1BEE0
:100FA000A308DBFA901A0F788C7B1AF1BEA308DB3A
:100FB000FA121011F1EE901A2922E493F622E64378
:100FC0008F01538FFDFFC3E583941C400122EF8501
:100FD00065B78566B7F0538FFE22438F02438F01BA
:100FE0008565B78566B7901A0DF0538FFC22901A6D
:100FF0000D7455F1BF901A0E74AAF1BF227A3079A0
:10100000D07820901A40120FBAE520F709A3DAF63B
:10101000227A3079D0901A40E7120FBF09A3DAF88C
:10102000227C05120345DCFB22C2AF1203541203DB
:101030005A12036012036612033912035412035A40
:1010400012036012036612033912035412035A1278
:101050000360120366D2AF22C2AF120366120360AE
:1010600012035A1203541203391203661203601258
:10107000035A120354120339120366120360120357
:071080005A120354D2AF2203
:1019FD00020B39100321FFFFFFFFFFFF09FF01FF5E
:101A0D0055AA01FFFFFFFFFF03FFFFFF25D0285061
:0D1A1D0004FF02FF7AFF0701FFFF0000FF3A
:101A4000234B5F485F323523202020202020202098
:101A500023424C48454C492445464D3842323123B7
:101A60002020202020202020202020202020202076
:101C0000C2AFC2D37597DE7597AD7581C075A90057
:101C100043FF80752438752503B1DB7529A5752A26
:101C2000F143F10153A4FED28075D4FF75E3407DEA
:101C3000FA780379E67C10752200752300901DE880
:101C40007B06752498752501308002814820800824
:101C5000D8FBD9F9DCF781BA308008D8FBD9F9DC98
:101C6000F781BAB19BE493A3C39A6004DDC381BA40
:101C7000DBDBB18D600281317B08E493FAA3B16EA6
:101C8000DBF87A30B16E752200752300B18DEAFC65
:101C9000EBFDC3ED94FE400EB18D8A278B28ED300D
:101CA000E0048A828B83B18D7AC270D8C3ED94FE32
:101CB000601950CEBD0029EC600F7520007521FF22
:101CC000752900752A000200008100A827A92808AC
:101CD00009D804D90281DDB191EAF281D10D81A642
:101CE000C3ED94035051EDA2E092007AC5C3E582A2
:101CF0009400E583941C508C200010438F02438F86
:101D0000018529B7852AB7F0300027A827A9280818
:101D100009438F01538FFDD804D902A132C3E58353
:101D2000941C4003A3A117E28529B7852AB7F0A325
:101D3000A117538FFC81827AC1BD030CE493A3FAEF
:101D4000B152DCF8B14A81828184AA22AB23B16E00
:101D5000EBFAEA6222752608C3E52313F523E52290
:101D600013F52250066323A0632201D526EAB1DBD6
:101D7000B1DB75260AEAF4200102D280300102C2EA
:101D800080B1DBC3134002C201D526EB22B191EA38
:101D9000FB208002A191308002A196752608AE2416
:101DA000AF25C3EF13FFEE13FEB1DFB1DBC3EA13C0
:101DB0003080024480FA30E703632201C3E5231335
:101DC000F523E52213F52250066323A0632201D5F3
:101DD00026D9E52265236523F52222AE24AF250E00
:101DE0000FDEFEDFFCD20122424C48656C693437BD
:061DF0003163E8B20601B8
:00000001FF
